:1000000000308A003D2D00000A108A100A11820774
:100010003F3406345B344F3466346D347D340734FA
:100020007F346F348034003439340830A10000004C
:1000300086128316861200008312BF0D0613031C5E
:1000400024288316061783120318292883160613FB
:100050008312831686168312861E2C28A10B17285E
:1000600000008612831686120000061700000000AA
:1000700086168312861E3A28A1010000061B211451
:1000800086128316861283120613831606138312B2
:10009000003483160617000086160000831206132C
:1000A000831606130000831286128316861203102D
:1000B0008312390D9038BA00BF001520EE30BF0012
:1000C000152083160613000086168312861E6628E6
:1000D00000006A2800008316061700008312390802
:1000E000BA000830BB008316061700008616000011
:1000F00083120613831606130000831286128316DA
:100100008612031083123A0D9038BC00BF001520F0
:10011000AC30BF0015203B08BF0015208316061326
:10012000000086168312861E932800009728000080
:1001300083160617000083128A115D2D0830BF0058
:100140002008C00083160617000086168312861E3C
:10015000A728061B0314061F0310A10D0000831619
:10016000861283128612BF0BA22883160617000080
:100170008312061340080319C0288316061383123E
:100180000000831686168312861EC428000086127D
:100190008316861200008312061383160613831239
:1001A000003483160617000086160000831206131B
:1001B000831606130000831286128316861203101C
:1001C0008312390D9038BE00BF001520AA30BF0041
:1001D0001520831606170000861600008312861E5F
:1001E000EF28061383160613000083128612831667
:1001F000861203108312390D9138BE00BF001520FE
:100200000130A0009E202108BA00A0019E202108F4
:10021000BB0083160613000086168312861E0E2965
:100220000000122900008316061700008312A301A4
:100230003A08BC002308BD003D08BF003C08BE00D2
:10024000C1010930C0001030C200A001A301BF0CE1
:10025000BE0C031C31294008A0070318A30A41085B
:10026000A307A30CA00CA20CA10CC20B27292208E7
:10027000BD002108BC00BB1F4A29BD1F4629043010
:10028000BC020030031C0130BD024A290430BC0707
:100290000318BD0A3D08BF003C08BE00C10105307F
:1002A000C0003F0841068039C300BF1F5C29BE095A
:1002B000BF09BE0A0319BF0AC11F6329C009C109CA
:1002C000C00A0319C10AA101A201A001A3014108AA
:1002D000031D6D294008031987291030C20003103F
:1002E000BE0DBF0DA00DA30D41082302031D7A29E9
:1002F00040082002031C83294008A002031CA3031A
:100300004108A3020314A10DA20DC20B6F29C31F44
:100310008E29A109A209A10A0319A20A20302107E6
:10032000BC002208BD000318BD0ABD1F9A29BD01EB
:10033000BC01A329BD1BA3293D08003C0318A32928
:10034000BD01FF30BC003C08A10000348E30A0008D
:100350003A08A1003908A200A301A108031DBA2987
:100360002208A100A2010830A002A108031DBA2999
:10037000A001C2290310A11BC129A20DA10DA00338
:10038000BA29A113003480308318BE06C301C4010A
:100390003A08C2003E08C20639080319B32AC10050
:1003A000A0003D080319BC2AC1020319582A031CE6
:1003B000162A3E08C700C7173F08C6004008C500F8
:1003C000C4010310C70CC60CC50CC40CC10BE0293A
:1003D000C21FED294314D02A4310411043163C306C
:1003E00084008313E52A4312C21B002A411C0B2AF6
:1003F000C70CC60CC50CC40CA00A0319CB2A0B2AC7
:10040000C71B0E2A0310C40DC50DC60DC70DA003D2
:100410000319CB2A002A4317782A43133A08C2004B
:10042000C21F142AC717C42AC713C42A3D08C10013
:10043000A0003908C1023A08C700C7173B08C60028
:100440003C08C500C4010310C70CC60CC50CC40C85
:10045000C10B222AC21F2F2AC314D02AC310411055
:10046000C316403084008313E52AC312C21B422AFC
:10047000411C4D2AC70CC60CC50CC40CA00A03199C
:10048000CB2A4D2AC71B502A0310C40DC50DC60D1B
:10049000C70DA0030319CB2A422AC317782AC31316
:1004A0003E08C200C21F562AC717C42AC713C42A4F
:1004B0003E08C700C7173F08C6004008C500C21F56
:1004C000652AC7134315D02A4311C40141103C309B
:1004D00084008313E52AC21B8E2A3A08C200411CFD
:1004E000782AC70CC60CC50CC40CA00A0319CB2A69
:1004F000C41F892AC50A031D892AC60A031D892A21
:10050000C70A031D892AC70CC60CC50CA00A03190B
:10051000CB2A431B0D2AC31B4F2AAD2A8030C706A6
:10052000C71F962AD02A3E08C200A32A3A08C20052
:10053000C708031DA32AC608031DA32AC508031D57
:10054000A32AA001C42AC71BAD2A0310C40DC50DE0
:10055000C60DC70DA00BA32ACB2AC21FB12AC717ED
:10056000C42AC713C42A3D08A0003E08C7003F089C
:10057000C6004008C500C42A3908A0003A08C700D0
:100580003B08C6003C08C5004708A1004608A20079
:100590004508A300032BA001A101A201A301032B85
:1005A000C401C509C609C709C409C40A031DDE2A56
:1005B000C50A031DDE2AC60A0319C70A4318EC2917
:1005C000C3182E2A4319642A932A0008C507031C5E
:1005D000EF2AC60A031DEF2AC70A03194114840330
:1005E0000008C607031CF72AC70A0319411484032D
:1005F0000008801F803AC70703184114431AF329E3
:10060000C31A352A6B2A00343D080319742BC50020
:1006100041080319742BC5070318152B7F30C50239
:10062000031C742B0319742B192B8130C507031875
:10063000742B4508A000A101A201A3013E08C90036
:10064000C9173F08C8004008C7001830C500C601D8
:10065000471C422B4408A307031C342BA20A031D8A
:10066000342BA10A0319C6174308A207031C3B2B0E
:10067000A10A0319C6174208BF00BF173F08A10708
:100680000318C617C60DA10CA20CA30CC90CC80CEC
:10069000C70C0310C50B272B0130A0070318742BC0
:1006A000A11B592BC90DA30DA20DA10DA003031968
:1006B000742BC91F6A2BA30A031D6A2BA20A031DF0
:1006C0006A2BA10A031D6A2BA10CA20CA30CA00A81
:1006D0000319742B3E08C6004208C606C61F722BBB
:1006E000A117782BA113782BA001A101A201A301CE
:1006F0000034410803193E2CCD00450803193E2C57
:10070000CD02031C882B7F30CD0703183E2C8E2B87
:100710008130CD02031C3E2C03193E2C4D08A00055
:10072000A101A201A301CC014208CB00CB174308D1
:10073000CA004408C9001930CD004808C90203188E
:10074000B12B0130CA020318B12BCB020318B12B15
:10075000CC020318B12BCC0ACB0ACA0A4808C90735
:10076000E32B4708CA020318CC2B0130CB02031835
:10077000CC2BCC020318CC2BCC0ACB0A4708CA07D7
:100780004808C907031CE32BCA0A031DE32BCB0A45
:10079000031DE32BCC0AE32B46088038CB02031859
:1007A000E22B0130CC020318E22BCC0A4608803839
:1007B000CB074708CA07031CC02BCB0A031DC02B5D
:1007C000CC0AC02B2314CD0BE62BF12B0310C90D43
:1007D000CA0DCB0DCC0D0310A30DA20DA10DCE0D96
:1007E0009D2B4E1CF92B0310A10CA20CA30CCE0CBC
:1007F000FC2BA00303193E2CCE1B252C0310C90D86
:10080000CA0DCB0DCC0D4808C9020318112C0130BC
:10081000CA020318112CCB020318112CCC02031CA2
:10082000342C4708CA0203181C2C0130CB020318D1
:100830001C2CCC02031C342C46088038CB02031835
:10084000252C0130CC02031C342CA30A031D342CAC
:10085000A20A031D342CA10A031D342CA00A03197B
:100860003E2CA10CA20CA30C4208CD004608CD06DC
:10087000CD1F3C2CA117422CA113422CA001A10199
:10088000A201A30100348E30A0003D08A0023E0862
:10089000A2003F08A100A217A00803195A2C0310B8
:1008A000A208031D562CA10803195A2CA20CA10C56
:1008B000A00B4F2CBE1F612CA109A209A10A03198C
:1008C000A20A00343B08A1013A0203186A2C3A0834
:1008D000A000762CA0010830BC00BA0DA00D3B088A
:1008E00020020318A000A10DBC0B6D2C00340830B1
:1008F000BC02031C872C3C30840083130310800C43
:1009000000080319872C852C0000800B842C0034F0
:100910002E08A3002D080420A10087008709831654
:100920000511831205112608B900B90AB903031984
:100930009D2CFF30BC007724962C2508BC00772422
:1009400083160511831205152C08A3002B0804201B
:10095000A100870087098316861383128613260851
:10096000B900B90AB9030319B92CFF30BC007724C8
:10097000B22C2508BC0077248316861383128617B1
:100980002A08A30029080420A100870087098316EC
:100990008512831285122608B900B90AB903031912
:1009A000D52CFF30BC007724CE2C2508BC00772442
:1009B0008316851283128516A708031DE52CA80847
:1009C000031DE52CA8010B30A7002808A300270869
:1009D0000420A100870087098316051283120512DF
:1009E0002608B900B90AB9030319FA2CFF30BC0074
:1009F0007724F32C2508BC00772483160512831274
:100A000005163008A3002F080420A10087008709DD
:100A100083168512831285122D302502B90026080F
:100A2000BA000030031C0130BA023A08BB00BB0A0E
:100A3000BB0303191F2DFF30BC007724182D390884
:100A4000BC00772483168512831285168A11BB2E6B
:100A5000393084008313000803193B2D0230A100B4
:100A6000A001A00B312DA10B302D9730A000A00BC1
:100A7000372D800B2E2D8A11C32E840183131F3036
:100A80008305713083168F000F08831203171F1020
:100A90009F101F119F1103131F13003003179E0097
:100AA00099019A0183169E0183129B0103138D12F3
:100AB0006430A500A601B901492803178D018316EA
:100AC0008C130C1483120C080313A601A500A508AF
:100AD000031D6D2DA6080319742DA608031D742D82
:100AE0002508FE3C0318772DA6013230A500B90178
:100AF000D120BA012108B900A6212308B400220898
:100B0000B3002108B2002008B10083143408BC00EF
:100B10003308BB003208BA003108B900C001BF0178
:100B2000BE018430BD00C3212008B9002108BA00ED
:100B30002208BB002308BC00C0002208BF00210817
:100B4000BE002008BD00C401C3012030C2008130B6
:100B5000C10004232008BD002108BE002208BF00F8
:100B60002308C000C4002208C3002108C2002008D6
:100B7000C100C801C7011030C6008230C50079230A
:100B80002308B8002208B7002108B6002008B500E5
:100B900003171F109F101F119F1103131F13003005
:100BA00003179E0003131F10941283168713061653
:100BB000061301308312940000308316940001085C
:100BC000C73908388100831290010030A1009200DB
:100BD0000030831692008312031799019A0183163D
:100BE0009E0183129B0103138D12713083168F00B7
:100BF0000F080730831287000030831687008312A6
:100C0000B901D120BA012108B900A6212308B400F6
:100C10002208B3002108B2002008B1008314340870
:100C2000BC003308BB003208BA003108B900C0016B
:100C3000BF01BE018430BD00C3212008B9002108D6
:100C4000BA002208BB002308BC00C0002208BF0075
:100C50002108BE002008BD00C401C3012030C2002D
:100C60008130C10004232008BD002108BE002208F5
:100C7000BF002308C000C4002208C3002108C2002E
:100C80002008C100C801C7011030C6008230C5006D
:100C900079232308B8002208B7002108B6002008ED
:100CA000B5003808C0003708BF003608BE00350858
:100CB000BD00C401C3012030C2008230C100042342
:100CC0002008B9002108BA002208BB002308BC0094
:100CD000C4002208C3002108C2002008C100C801C6
:100CE000C7014830C6008530C50079232308C000FD
:100CF0002208BF002108BE002008BD0043242208AE
:100D0000A8002108A7003808C0003708BF0036082F
:100D1000BE003508BD0043242108BA000A30BB00DC
:100D20006224AA012008A9003808C0003708BF00C3
:100D30003608BE003508BD00C401C3012030C20022
:100D40008230C10004232308C0002208BF0021080C
:100D5000BE002008BD0043242108BA000A30BB00B1
:100D60006224AC012008AB00AE010C30AD00B00134
:100D70000A30AF00882C831606168312061AF12E4D
:100D80009630B900282D3230A5070318A60A260888
:100D9000023C0318D52EFF3A031DD22E2508E73C4E
:100DA0000318D52EA6013230A50003178D010313B9
:100DB000250803178C0083168C130C15831203135C
:100DC0000B08A0008B138316031755308D00AA3033
:100DD0008D008C148C18EA2E0C118312031320083A
:080DE0008B048316F92D63005A
:02400E00843CF0
:00000001FF
